:100000000C943F030C9477030C9477030C947703C0
:100010000C9477030C9477030C9477030C94770378
:100020000C9477030C9477030C9429180C94DE1627
:100030000C94C3190C9477030C9477030C947703F6
:100040000C9477030C9477030C9477030C94770348
:100050000C9477030C9482190C9477030C94770317
:100060000C9477030C9477030C9477030C94770328
:100070000C9477030C9477030C9477030C94770318
:100080000C9477030C9477030C9477030C94770308
:100090000C9477030C9477030C9477030C947703F8
:1000A0000C9477030C9477030C94770383048804EF
:1000B000A104AA04B504BC04C804CF04440744073F
:1000C00076077607E8079009900990090408E20886
:1000D000F308F308990BB30BDE0B1A0C550C940CB8
:1000E000D80CDB0CE10CE40CE70CEA0CED0CF00C8A
:1000F000F30CF60CF90CFE0C010D040D090D4D0D61
:10010000910DD90DDC0DE10D4C0E310F771E9E1EA9
:1001100036209E1E3620E61E091F3620F81F0B20B3
:10012000002445550025355600263646002737471A
:100130000028384800293949002A3A4A002B3B4B0D
:1001400000A4948400A5958500A7978700A89888A7
:1001500000A9998900AA9A7900AB8A7A002C4D5D92
:10016000002D3D5E002E3E4E002F3F4F0030405090
:10017000003141510032425200334353006C5C7CE9
:100180000073638300AC9C8C00AD9D8D00AE9E8E91
:1001900000AF9F8F00B0A09000B1A19100B2A281EA
:1001A00000B3928201244555012535560126364675
:1001B000012737470128384801293949012A3A4A95
:1001C000012B3B4B01A4948401A5958501A696863D
:1001D00001A7978701A8988801A9998901AA9A7906
:1001E00001AB8A7A012C4D5D012D3D5E012E3E4E04
:1001F000012F3F4F013040500132425201334353EF
:1002000001AC9C8C01AD9D8D01AE9E8E01AF9F8F88
:1002100001B0A09001B1A19101B2A28101B392827B
:1002200005010980A101850319012AB700150126DE
:10023000B700950175108100C0050C0901A1018569
:100240000419012AA002150126A00295017510814A
:1002500000C005010906A1018506050719E029E787
:10026000150025019508750181020507190029EF80
:100270001500250195F07501810205081901290570
:10028000950575019102950175039101C00501095C
:1002900006A101050719E029E71500250195087554
:1002A0000181029501750881010507190029FF15D3
:1002B0000026FF009506750881000508190129052B
:1002C000950575019102950175039101C009023BE5
:1002D00000020100A0FA0904000001030101000965
:1002E00021110100012240000705810308000109D6
:1002F0000401000103000000092111010001226D29
:10030000000705820320000112010002000000081E
:100310004E693653010001020001120353005100DF
:1003200055004100520045002E00580000001A03FD
:1003300069004E0045005400540020005300740032
:100340007500640069006F000000040309040004E4
:100350007F3F1F643214643214783C1E1E140A0559
:100360002223252628292A2C2D2F303233353638C2
:100370003A3B3D3E4042434547494A4C4E5051531B
:100380005557595A5C5E6062646668696B6D6F713F
:10039000737577797B7D7F81838587898A8C8E9041
:1003A000929496989A9C9E9FA1A3A5A7A8AAACAE4A
:1003B000AFB1B3B4B6B8B9BBBCBEBFC1C2C3C5C68A
:1003C000C7C9CACBCCCDCED0D1D2D2D3D4D5D6D733
:1003D000D7D8D9D9DADADBDBDBDCDCDCDCDCDDDD71
:1003E000DDDDDCDCDCDCDCDBDBDBDADAD9D9D8D761
:1003F000D7D6D5D4D3D2D2D1D0CECDCCCBCAC9C703
:10040000C6C5C3C2C1BFBEBCBBB9B8B6B4B3B1AF39
:10041000AEACAAA8A7A5A3A19F9E9C9A98969492D9
:10042000908E8C8A89878583817F7D7B79777573B0
:10043000716F6D6B6968666462605E5C5A5957558E
:100440005351504E4C4A4947454342403E3D3B3A4A
:100450003836353332302F2D2C2A292826252322D1
:100460000001010101010101010102020202020277
:10047000020202030303030303030304040404044A
:100480000404050505050506060606060707070711
:100490000708080808090909090A0A0A0B0B0B0CC6
:1004A0000C0C0D0D0D0E0E0E0F0F0F101011111163
:1004B00012121313141415151616171718181919E4
:1004C0001A1A1B1B1C1D1D1E1E1F20202122222349
:1004D0002424252626272829292A2B2C2D2D2E2F8A
:1004E00030313232333435363738393A3B3C3D3EA1
:1004F0003F404142434445464748494A4C4D4E4F90
:1005000050515354555658595A5B5D5E5F61626451
:10051000656668696B6C6D6F7072737577787A7BDE
:100520007D7E8082838587888A8C8E8F9193959635
:10053000989A9C9EA0A2A3A5A7A9ABADAFB1B3B555
:10054000B7BABCBEC0C2C4C6C9CBCDCFD1D4D6D831
:10055000DBDDDFE2E4E7E9EBEEF0F3F5F8FAFDFFCF
:10056000FFAA7F554029001E001F00200021002205
:100570000023002500260027002D002E004C002A15
:10058000002B0014001A000800150017001C0018AA
:10059000000C00120013002F00300031003900045D
:1005A000001600070009000A000B000D000E000FE6
:1005B000003300340000002800E10000001D001B93
:1005C0000006001900050011001000360037003841
:1005D00000E5004D00E000E300E200000000000044
:1005E000002C002400000000000000E6000151E49F
:1005F0000001003A003B003C003D003E003F00414E
:1006000000420043004400450001004600005CC376
:100610005CC45C01006B006C000100010001000182
:100620000001004B004E000100010001000100012B
:1006300000010001005000510052004F004A004DDF
:1006400000000001000100000001000100010001A4
:100650000001000100010001000100010001000192
:100660000001000100010000000000000001004046
:100670000000000000000001000100010000112442
:100680001FBECFEFDAE0DEBFCDBF04B603FE18C059
:1006900080917F0690918006A0918106B09182069C
:1006A0008730904BA740B04B59F410927F061092C0
:1006B00080061092810610928206E0E0F8E3099528
:1006C00012E0A0E0B1E0E6E1F0E602C005900D9294
:1006D000A23AB107D9F726E0A2EAB2E001C01D9222
:1006E000AF37B207E1F70E945E200C9409300C94FA
:1006F00000001F93CF93DF93CDB7DEB767970FB698
:10070000F894DEBF0FBECDBF4B8B5C8B6D8B7E8BA9
:100710008F8B61111092340486E09E01235F3F4F5E
:10072000D901E82F1D92EA95E9F795E0FE0173964D
:10073000D90101900D929A95E1F79C894E895F89C4
:100740007B897D879E876F87598B488BF901DE01F6
:10075000179601900D928A95E1F7CE0107960E94B7
:100760007A1381113EC086E0FE013796DE011196B4
:1007700001900D928A95E1F7FF81E8856A857B8576
:100780006115710531F0EF3F31F481E0FF3F19F45D
:1007900003C081E001C080E080FD23C02091E1031F
:1007A00030E0C9010196877099274091120450E00A
:1007B0008417950779F1F983EA837D836C8396E04A
:1007C000929FD001939FB00D1124AE51BC4FFE01FA
:1007D000319601900D929A95E1F78093E1030E9482
:1007E000041316E0809112049091E1038917F9F047
:1007F000189FC00111248E519C4F0E947A138823A8
:10080000B1F08091120490E001968770992780934F
:100810001204E8CF0E94812B1092E103109212047F
:10082000EBEDF3E086E0DF011D928A95E9F767962C
:100830000FB6F894DEBF0FBECDBFDF91CF911F91F1
:1008400008958F929F92AF92BF92CF92DF92EF92D4
:10085000FF920F931F93CF93DF93CDB7DEB72A9705
:100860000FB6F894DEBF0FBECDBFFC010081D18072
:1008700083819481892B39F01FEFD11206C091E05A
:100880000F3F19F403C091E001C090E090FD73C6E2
:100890007F0185E0DE01169601900D928A95E1F7C1
:1008A000F70122818E819F81222349F00E943B2AF9
:1008B000182F682F8E819F810E94DC2A03C00E941E
:1008C000B02A182F26E4129FF00111243EE0D39E97
:1008D000E00DF11D1124E00FF11DEE0FFF1FEB598C
:1008E000FA4F05911491F7018281882309F462C0BF
:1008F000F801EB56F109E830F10508F05BC0EA5A5F
:10090000FF4F0C94CE2F9091E60581E089270FC010
:100910009091E605892F869586958F5F8C3108F03A
:1009200081E0937009F450C5880F880F892B80935C
:10093000E605109206018091E50581608093E5054A
:1009400043C58091E70590E04091E9056091E80595
:10095000089608C08091E70590E04091E905609114
:10096000E80508970E94CB1B2FC56091E80520E1A0
:10097000620F08F46FEF06C06091E80520E1621B8A
:1009800008F460E08091E7054091E90590E0EACF46
:100990004091E90520E1420F08F44FEF06C0409175
:1009A000E90520E1421B08F440E08091E7056091F1
:1009B000E805ECCF043F2CE5120799F406E221EE9E
:1009C00040EE64EF7CE509C0083DFCE51F0711F52A
:1009D00006E221EE41EE68ED7CE5C7010E94811A36
:1009E000F3C4053F3CE5130708F05CC1093D9CE5F5
:1009F000190731F407E225EE45EE69ED7CE5EDCF10
:100A00000A3DECE51E0701F708E221E045EE6AED3C
:100A10007CE5E3CF882309F47AC11092A105043064
:100A2000FDE51F0758F40B3F2CE5120780F4C801C1
:100A300082509C45449708F054C109C002363DE5F8
:100A4000130729F0063A8DE5180709F04AC10E94FC
:100A5000EC119093AE058093AD0501319CE519072B
:100A600009F4C6C008F042C00930FCE51F0709F4CC
:100A70009BC000F505303CE5130709F485C078F408
:100A800003309CE5190709F478C008F07AC00230F9
:100A90001C4509F0F7C08091AD058160F1C00730B9
:100AA0002CE5120709F478C008F07AC08091AD05F2
:100AB0008061E6C00D308CE5180709F487C058F452
:100AC0000B30ECE51E0709F479C008F07BC080917B
:100AD000AD0588606FC00F302CE5120709F480C0A7
:100AE00008F082C08091AD05877FCAC00E3F8CE5BB
:100AF000180709F471C000F50531ECE51E0709F48B
:100B000085C068F403312CE5120709F475C008F0BC
:100B100095C00E94812B8091AD058F77B1C00C3FAD
:100B20008CE51807A9F108F054C00B3F1C4509F0EB
:100B3000A9C08091AE0540C00230FDE51F0709F451
:100B400089C058F401153DE5130709F45AC008F0AF
:100B500069C08091AE0582602FC002369DE51907FD
:100B600009F47EC0063AEDE51E0709F483C00330A0
:100B70001D4509F087C060E06EC08091AD058260C0
:100B80007FC08091AD0516C08091AD05886078C0AA
:100B90008091AE0582604FC08091AD05806270C0CB
:100BA0008091AD0580646CC00E94812B8091AD0561
:100BB000806866C0846064C081603DC08091AD057E
:100BC0008E7F5EC08091AD058D7F5AC08091AD054E
:100BD00016C08091AE0518C08091AE058D7F2BC0E8
:100BE0008091AD058F7E4CC08091AD058F7D48C052
:100BF0008091AD058F7B44C08091AD05877F8B7F51
:100C00003FC08091AE058D7F8E7F15C08091AD0570
:100C100082FB222720F991E0922790FB82F990FB3A
:100C200083F92EC08091AE05982F909591708E7F9C
:100C3000892B90FB81F98093AE0524C00E94812B03
:100C40008091AD0587FB222720F991E0922790FB48
:100C500087F916C061E08EE090E00E94252F12C057
:100C60008091AD0584FB222720F991E0922790FB2B
:100C700084F906C08091AD05982F909590FB80F97E
:100C80008093AD056091AD051091AE0584E090E0D4
:100C90000E94252F612F82E290E00E94252F0E9462
:100CA000812B92C3063F2CE5120731F406E221EEB8
:100CB00042EE66EF7CE591CE063F3CE5130730F44B
:100CC00007E225EE44EE65EF7CE587CE073F9CE525
:100CD000190709F09FCE07E225EE46EE67EF7CE5A7
:100CE0007CCE0631ECE51E0721F5809135048A7A29
:100CF00091E009F490E09093A402882311F065E359
:100D000001C069E28BEB93E00E94141A0FC0063118
:100D1000FCE51F0709F040C08091A402882309F474
:100D200076C365E38BEB93E00E94EC190E94751289
:100D30004BC30B353DE5130749F158F401159CE50C
:100D40001907B1F00F3D1C4509F042C00E94FD118A
:100D50003BC30C35FDE51F07D9F00D351D45C1F529
:100D60008091AE0582FB882780F991E0892711C028
:100D70000E94812B3FEF84E39CE031508040904003
:100D8000E1F700C000000E945E191EC381E001C0AF
:100D900080E00E94E7121CC08091350482720D3CF5
:100DA0002CE5120709F4C7C308F0F7C2073C9CE51D
:100DB000190709F4ACC308F03AC3043CFCE51F076B
:100DC00009F49BC308F025C3033C1C4509F470C318
:100DD000F70182810081D180882359F0802F9D2DD9
:100DE0000E943B2A182F682F802F9D2D0E94DC2AFD
:100DF00005C0802F9D2D0E94B02A182F26E4129F37
:100E0000F00111243EE0D39EE00DF11D1124E00F0E
:100E1000F11DEE0FFF1FEB59FA4F859194910E943F
:100E200063108C01982EF701D280A580A2943FE038
:100E3000A322809113048770B9F0DD20A9F0812FDF
:100E4000807F803421F080E2800F883068F08091CC
:100E5000AE0582FD09C082E00E94CA12809113048F
:100E60008770CC24C3948111C12CB12EB2949FE021
:100E7000B9228B2D90E08C30910508F051C2FC0115
:100E8000E25AFF4F0C94CE2F812F807F1F70882352
:100E900011F01295107FDD20B9F0112309F42DC255
:100EA00080E2800F883010F0911006C080913504E8
:100EB000182B1093350405C080913404182B10931F
:100EC00034040E94751219C2802F0E94A72B11238F
:100ED00009F426C2005E083078F1992069F1109576
:100EE0008091340418231093340429C0812F807F0B
:100EF0001F70803211F01295107F992021F0F1E0DF
:100F00009F16D9F149C08091AE0582FF1BC0DD203C
:100F100069F0112339F080913504182B10933504B2
:100F20000E94751280E00E94D12BFAC180E00E94DD
:100F3000A72B112309F4F4C1812F0E946E120E9485
:100F40007512EEC1DD2081F080913604AA2051F0A7
:100F500001E0A01207C0182B181709F4E1C1109383
:100F60003604DEC1812B10C0AA2021F021E0A21698
:100F700009F4D6C10E94681227C0DD2041F035E097
:100F80003A1508F4CDC1812F0E949D2BC9C184E080
:100F90008A1508F4C5C118C0DD2049F0AA2099F3CC
:100FA000F701858180FFA9C18F708583ECCFAA20CE
:100FB00059F0093309F0B1C1FFEF17EE23E0F1500A
:100FC00010402040E1F7A7C1812F0E94962BA8C1B5
:100FD000812F86958695837019F0813059F0A0C1D4
:100FE000DD2019F0C801937002C080E090E00E94FB
:100FF0005F1A9CC1DD2019F0C801937002C080E027
:1010000090E00E94491A92C1812F837009F069C053
:10101000D1108AC1902F929596959770990F990F3C
:10102000802F8F70882E912CA12CB12C092E04C0FA
:10103000880C991CAA1CBB1C0A94D2F704FF12C08E
:101040004FE050E060E070E004C0440F551F661FA1
:10105000771F9A95D2F7DB01CA0180959095A095EC
:10106000B09503C080E090E0DC0116951695412F05
:101070004370423019F1C8F40091370410913804DC
:101080002091390430913A04413059F08829992946
:10109000AA29BB29BC01CD0160237123822393239C
:1010A0000AC0802A912AA22AB32ABC01CD0168294C
:1010B00079298A299B290E94572B36C18829992989
:1010C000AA29BB29009137041091380420913904D2
:1010D00030913A04BC01CD01602771278227932704
:1010E000EACFDD2019F0812F817001C08695882319
:1010F00009F41AC1902F929596959770990F990FB0
:10110000802F8F70882E912CA12CB12C092E04C019
:10111000880C991CAA1CBB1C0A94D2F704FF12C0AD
:101120004FE050E060E070E004C0440F551F661FC0
:10113000771F9A95D2F7DB01CA0180959095A0950B
:10114000B09503C080E090E0DC0116951695412F24
:1011500043704230D9F068F50091F6051091F7051B
:101160002091F8053091F905413059F088299929E5
:10117000AA29BB29BC01CD016023712382239323BB
:101180001EC0802A912AA22AB32A13C0882999292D
:10119000AA29BB290091F6051091F7052091F805C1
:1011A0003091F905BC01CD01602771278227932773
:1011B00006C0BC01CD01682979298A299B290E9492
:1011C000072BB2C01F70DD2039F0812F0E94362B13
:1011D000802F0E949D2BA8C0802F0E94962B812FCC
:1011E0000E94112BA1C0802F32EF931609F443C047
:1011F000391538F090EF991659F0E1EF9E16B1F1DC
:1012000077C0F3EF9F16F1F124EF921659F170C0F9
:10121000DD2019F134E03A1508F482C01F7181E035
:1012200090E0A0E0B0E0AC01BD0104C0440F551F48
:10123000661F771F1A95D2F78091F6059091F705F2
:10124000A091F805B091F9058A019B01082719279B
:101250002A273B27C901B80129C025E02A1508F42F
:101260005FC0DCCF8091AE0582FF23C0DD2029F076
:10127000812F8F7130C0DD20D9F3812F8F710E94B3
:10128000112B4EC0DD2079F01F7181E090E0A0E0CD
:10129000B0E0BC01CD0104C0660F771F881F991F05
:1012A0001A95D2F703C060E070E0CB010E94072BD3
:1012B00037C0DD2099F01F71812F0E94362B80915D
:1012C000AE0582FD07C038E0139FC0011124836082
:1012D00080931304812F0E94362B22C081E00E944C
:1012E000CA1281E08A15E0F482E00E94CA1218C096
:1012F000DD2029F0AA2009F4BBCF802F14CEAA202C
:1013000009F4BBCF893349F49FEFE7EEF3E0915046
:10131000E040F040E1F700C00000802F0E94A72BC2
:1013200088EF8B0D843010F40E94751ACC20A9F040
:101330008091130480FD11C0F70112828595859577
:1013400085950E94362BC7010E94210480911304C9
:101350008595859585950E94112B85E0F701DE0125
:10136000119601900D928A95E1F789819A810E94E8
:10137000B02A9A8106E4809FF00111241EE0919F1B
:10138000E00DF11D11248981E80FF11DEE0FFF1F03
:10139000EB59FA4F85919491EEC0023D2CE512076E
:1013A00009F4D9C008F465C0053D2CE5120709F41D
:1013B000D8C008F471C0063DECE51E0709F4D6C09C
:1013C0000E351D4509F004CD80911304877009F492
:1013D000D2C0F7018281882309F4CDC08091AE0587
:1013E00082FDC9C082E02A960FB6F894DEBF0FBE18
:1013F000CDBFDF91CF911F910F91FF90EF90DF90C4
:10140000CF90BF90AF909F908F900C94CA1269E2DA
:1014100089CC053C9CE5190709F474C0063C1C45C1
:1014200009F0D6CC48EC59E261ED79E288C00A3C7B
:10143000FCE51F0709F475C070F4083C3CE5130790
:1014400009F46AC0093C1C4509F0C2CC4CEB59E2D6
:1014500060EB79E274C00B3CECE51E0709F466C052
:101460000C3C1C4509F0B4CC49E058E26AE178E252
:1014700066C00F3C8CE5180709F467C008F462C029
:10148000003DECE51E0709F463C0013D1C4509F071
:101490009FCC6EE089E067C0033D8CE5180709F436
:1014A0005DC0043D1C4509F093CC61E088E160C05B
:1014B00080919A0580FF1BC08E7F80939A05609172
:1014C0009A0570919B0580919C0590919D050E94C5
:1014D000F727109251060FEF10E722E0015010405D
:1014E0002040E1F700C000000E9496276DCF816088
:1014F00080939A0561E086953BC04CE15AE265E233
:101500007AE21DC045E25AE26CE17AE218C041ED90
:1015100059E268EC79E213C040EB59E26CEB79E2F6
:101520000EC048E959E264EA79E209C044EA59E2A6
:1015300068E979E204C04AE158E269E078E20E9491
:101540001E1B42CF61E081E013C065E082E00BC06A
:1015500068E086E008C064E18FE005C067E185E1EE
:1015600002C062E289E10E940C1B2ECF61E083E29F
:101570000E94DA2929CF2A960FB6F894DEBF0FBE53
:10158000CDBFDF91CF911F910F91FF90EF90DF9032
:10159000CF90BF90AF909F908F9008955F926F9281
:1015A0007F928F929F92AF92BF92CF92DF92EF92F3
:1015B000FF920F931F93CF93DF938FB7F8944091CF
:1015C000A9055091AA056091AB057091AC058FBF3C
:1015D0004093A5025093A6026093A7027093A802BD
:1015E0008091E605982F937021F0D82FD695D69547
:1015F00001C0D0E090910601913091F028F0923036
:1016000091F19330D9F1F3C4109208014093E105B0
:101610005093E2056093E3057093E40581E02BC0ED
:1016200090910501D9130CC0837090E040910401A2
:1016300050E021E08417950709F420E0822F01C0D3
:1016400081E0817080930A018091EB0590910901FE
:10165000981709F440C08093090140E060E080E001
:101660000E94A62638C0D0930501837080930401A0
:101670000E94442C83E080930601B9C48091E50563
:10168000882351F046E050E06CE170E086EE95E092
:101690000E94152F1092E5054091E1055091E20559
:1016A0006091E3057091E4052FB7F8948091A90546
:1016B0009091AA05A091AB05B091AC052FBF841BFA
:1016C000950BA60BB70B4097A105B10508F48FC485
:1016D000109206018CC48D2F90E08C319105F0F1B1
:1016E000809108018F5F8093080182E0809306015A
:1016F00080910A0181112EC0DD2309F4BBCF0E9425
:10170000751A81FF74C420E040E06FEF88E090E03C
:10171000DF91CF911F910F91FF90EF90DF90CF90CD
:10172000BF90AF909F908F907F906F905F900C9440
:10173000A82680910A01882329F040E060E080E03B
:101740000E94A626C0E0809108018F5F8093080167
:10175000CC2359F2DD2309F44AC4D1CFFC01E65968
:10176000FF4F0C94CE2F80910801CDE08C9FC02DAF
:1017700011241DE01C0F113408F010E46091E705FE
:101780007091E8058091E9050E943B28062FF72E0D
:10179000E82EC11708F008C2EC2FF0E0DF01AF5DC2
:1017A000BD4F8C9190910901982331F02E2D402F3F
:1017B0006F2DCF010E94A826CF5FEBCFC09108010B
:1017C0008DE0C89FC02D11241DE01C0F113408F0BE
:1017D00010E4F090E8050091E905E090E705B70115
:1017E000802F0E943B28D62EC72EB82E6091EA0586
:1017F0006E0D7F2D802F0E943B28062FF72EE82E9E
:10180000C11708F0D1C18C2F90E0FC01EF5DFD4FB6
:10181000308120910901232359F030FF04C02E2D7F
:10182000402F6F2D03C02B2D4D2D6C2D0E94A8260F
:10183000CF5FE6CFC09108018DE0C89FC02D112475
:101840001DE01C0F113408F010E4D090E805C090A2
:10185000E9052091EA0500E4029F012D1124C1173A
:1018600008F0A2C1EC2EF12CF701EF5DFD4F908145
:10187000809109018923B9F0F701EE0FFF1FEE55A2
:10188000FE4F808182958F706091E705809F600D8B
:1018900011247D2D8C2D0E943B28462F282F672F49
:1018A000C7010E94A826CF5FDACFC09108018DE062
:1018B000C89FC02D11241DE01C0F113408F010E446
:1018C000D090E805C090E9052091EA0500E4029F68
:1018D000012D1124C11708F067C1EC2EF12CF7017E
:1018E000EF5DFD4F9081809109018923D9F0F701C7
:1018F000EE0FFF1FEF55FE4F6081069FB0011124D0
:1019000045E0759567954A95E1F78091E705680F81
:101910007D2D8C2D0E943B28462F282F672FC70135
:101920000E94A826CF5FD6CFC09108018DE0C89F46
:10193000C02D11241DE01C0F113408F010E4F090AC
:10194000E7050091E805E090E9056091EA056695F4
:10195000669566958091E1059091E2050E94792750
:101960000E94C526805887FD8195880F282F3E2D1F
:10197000239F212D1124822F6F2D702F0E943B2831
:10198000062FF72EE82EC11708F00EC1EC2FF0E05D
:10199000DF01AF5DBD4F8C9190910901982331F02B
:1019A0002E2D402F6F2DCF010E94A826CF5FEBCFA9
:1019B0008EEC93E203C18CE694E20E94091DC82FCD
:1019C000C2CE81E594E217C08CEC93E2F7C083ECC1
:1019D00093E2F4C08AEB93E2F1C08FE993E2EEC0A8
:1019E00080E993E208C080E597E2E7CF80E494E2E3
:1019F000E4CF8CE294E20E948D1CE1CF82E693E278
:101A000005C080E393E202C082EF92E20E942C1CA8
:101A1000D6CF80910A0181111EC06091EA0520E1B4
:101A2000620F08F46FEF8091E1059091E2050E944A
:101A300079276AE070E00E94782E892B09F082CE27
:101A40000E94D82E60E470E00E94BA2F60910901D4
:101A50000E94542D77CE809108010DE0809F002DCB
:101A600011242DE0F22EF00E80E48F1510F490E496
:101A7000F92E10E0CF2CD12C0C151D0544F46091EB
:101A80000901C8010E94542D0F5F1F4FF5CFC1E01F
:101A9000EFE3EF1508F057CE55CE80910A01811182
:101AA0001EC06091EA0520E1620F08F46FEF80919B
:101AB000E1059091E2050E94792765E070E00E94BF
:101AC000782E892B09F03ECE0E94D82E60E470E07B
:101AD0000E94BA2F609109010E942D2D33CE809172
:101AE00008010DE0809F002D11248DE0F82EF00EEE
:101AF000F0E4FF1510F410E4F12E10E0CF2CD12CFF
:101B00000C151D0544F460910901C8010E942D2D9A
:101B10000F5F1F4FF5CFC1E02FE32F1508F013CE55
:101B200011CEC09108018DE0C89FC02D11241DE089
:101B30001C0F113408F010E4F090E8050091E9055D
:101B4000E090E7056091EA05669566956695809157
:101B5000E1059091E2050E9479270E94C5268058F0
:101B600087FD8195880F682F2CE0629F612D1124DD
:101B70006E0D7F2D802F0E943B28062FF72EE82E1A
:101B8000C11790F4EC2FF0E0DF01AF5DBD4F8C91F9
:101B900090910901982331F02E2D402F6F2DCF0108
:101BA0000E94A826CF5FECCFC1E0103408F4CBCD63
:101BB000C9CD86EE96E202C081EE92E20E94DE1B63
:101BC000FECE4091A9025091AA026091AB027091A1
:101BD000AC028091E1059091E205A091E305B091FE
:101BE000E40584179507A607B70708F4ABCD0E9454
:101BF0000A27C82F0E940A2790E4891BF0F7890F53
:101C0000082F10E0F801EF5DFD4F909109018081F0
:101C1000892309F4EAC1C1FF04C020E040E060E08C
:101C200013C00E940A27C82F0E940A278695782F82
:101C30002FE7720F08F47FEF6C2F8091E9050E9467
:101C40003B28462F282F672FC8010E94A8262091E5
:101C5000EA0530E1230F08F42FEF60E1822F90E0D6
:101C60000E947927BC0184EF91E00E94782E809138
:101C7000E1059091E205A091E305B091E405860F9E
:101C8000971FA11DB11D8093A9029093AA02A09352
:101C9000AB02B093AC0256CD40916D0350916E03F0
:101CA00060916F03709170038091E1059091E2055E
:101CB000A091E305B091E40584179507A607B7073F
:101CC00008F440CD80910A0181110DC08091080176
:101CD000CDE08C9FC02D11240DE00C0F013408F4D1
:101CE00054C000E452C040E060E080E00E94A626BC
:101CF000CDEAEC2EC2E0FC2E00E010E0CFE70E941F
:101D00000A2781FF05C0F7011082118212821DC0CF
:101D10000E940A27B82E0E940A278695782F2C2F1A
:101D2000720F08F47FEFC801880F991F800F911F71
:101D3000FC01E355FD4F6F016B2D8091E9050E9479
:101D40003B28F6016083718382830F5F1F4FF3E0AE
:101D5000EF0EF11C0034110591F6B8CF8C2F90E0F6
:101D6000FC01EF5DFD4F308120910901232361F0DB
:101D7000FC01EE0FFF1FE80FF91FE355FD4F228115
:101D8000408161810E94A826CF5FC01738F3C1E06F
:101D9000003408F0C0E0003408F4D5CC20E010E0B6
:101DA00001501109822F90E080179107CCF4AC010B
:101DB000440F551F480F591F43555D4F0196FC01B5
:101DC000EE0FFF1F8E0F9F1FFC01E355FD4F80811B
:101DD0009181A281FA0180839183A2832F5FE2CF58
:101DE0000E940A277801EE0CFF1C81FF09C00E0D2E
:101DF0001F1DF801E355FD4F10821182128218C099
:101E00000E940A27D82E0E940A278695782F2FE74E
:101E1000720F08F47FEF0E0D1F1D03551D4F6D2D22
:101E20008091E9050E943B28F801608371838283D9
:101E30000E9483270091E1051091E2052091E305BE
:101E40003091E405DC01CB01800F911FA21FB31F6D
:101E500080936D0390936E03A0936F03B093700310
:101E600072CC4091B7035091B8036091B90370915F
:101E7000BA038091E1059091E205A091E305B0914C
:101E8000E40584179507A607B70708F45BCC809193
:101E90000A01882329F040E060E080E00E94A62645
:101EA0006091E7057091E8058091E9050E943B2863
:101EB000C62F772E682E91E7E92E93E0F92E0BE5D9
:101EC00011E021EAA22E21E0B22E4701C12CD12C33
:101ED000F4018081F801EC0DFD1D882329F080813B
:101EE000262D4C2F672D04C0808120E040E060E06B
:101EF00090E00E94A826F401818181934F01FFEFB9
:101F0000CF1ADF0A26E0C216D10411F74801670193
:101F10008DE0582EF6018585F401882329F085850A
:101F2000262D4C2F672D04C0858520E040E060E021
:101F300090E00E94A826F601848585875A94F1E0F6
:101F4000CF1AD10821E0821A910837E05312E2CF6C
:101F5000F7018781F801882329F08781262D4C2FEE
:101F6000672D04C0878120E040E060E090E00E949F
:101F7000A826F7018681F801882329F08681262D7D
:101F80004C2F672D04C0868120E040E060E090E0A7
:101F90000E94A8260E940A27837091E009F090E031
:101FA000F70196839783FEE0EF0EF11C025F1F4F4F
:101FB000A016B10609F089CF0E9483270091E105A0
:101FC0001091E2052091E3053091E405DC01CB019D
:101FD000800F911FA21FB31F8093B7039093B80384
:101FE000A093B903B093BA03ADCBC1E0ACCBDF9102
:101FF000CF911F910F91FF90EF90DF90CF90BF9006
:10200000AF909F908F907F906F905F90089580E049
:1020100008959091AD0592FF0DC0282F28712830AA
:1020200019F4877F846006C0282F2471243011F4AE
:102030008B7F886093FF0DC0282F2871283119F4F9
:10204000877E846106C0282F2471243111F48B7E91
:1020500088612091AE0520FF0DC0382F38713830CF
:1020600019F4877F816006C0382F3171313011F447
:102070008E7F886021FF0DC0282F2871283119F428
:10208000877E816106C0282F2171213111F48E7E57
:10209000886194FD877E0895F894E82FE295EF70AB
:1020A000F0E031A1282F2F7081E090E001C0880F6F
:1020B0002A95EAF7982F9095932391A392A1892BC3
:1020C00082A378940895CF93DF938238910569F1C4
:1020D000B0F48133910509F46FC048F48932910559
:1020E00009F465C08A32910509F46BC08AC0853352
:1020F000910509F457C089339105B9F082C0833E38
:10210000910571F138F4803E9105B1F0823E910560
:1021100011F177C0863E9105B9F1873E9105C9F16D
:10212000843E910509F06DC024C02091AD0520FDCD
:1021300053C021FD51C065C08091AD0580FD46C0F2
:102140008091AE0580FF48C08091AD0584FD3FC100
:1021500083EE90E03EC18091AD0582FF3AC0F4CF9E
:102160008091AD0582FD35C08091AE0580FD34C003
:10217000EBCF8091AE0581FF35C08091AD0584FD28
:1021800026C187EE90E025C18091AD0583FF27C071
:10219000F4CF8091AD0583FD22C08091AE0581FD15
:1021A00021C0EBCF8091AD0585FD1FC021C080917E
:1021B000AD0585FD1DC019C08091AD0586FD1BC014
:1021C0001DC08091AD0586FD19C015C089E390E062
:1021D00000C182EE90E0FDC080EE90E0FAC086EE95
:1021E00090E0F7C084EE90E0F4C089E290E0F1C0A6
:1021F00085E390E0EEC08AE290E0EBC081E390E0FE
:10220000E8C0811532E5930708F069C0811541E502
:10221000940728F0982F8827816F906ADAC0883E4B
:10222000910568F5803E910508F0D3C0883A910584
:10223000B8F4853A910548F0855AE82FF0E0E65D5C
:10224000FE4F808190E09064C4C08130910509F414
:10225000BBC008F4BCC08430910508F4B8C0B9C054
:102260008F3B910508F0B3C0885AE82FF0E0EE0FDD
:10227000FF1FE35DFE4F808191819464AAC08115A8
:1022800020E59207F0F09C0174E0369527957A9549
:10229000E1F7922F9370482F437021E030E002C0A5
:1022A000220F331F4A95E2F73C68392B8F70982F25
:1022B0009695969540E2949FC0011124822B932B12
:1022C00088C0811530E4930718F09F70906A81C030
:1022D0009C013A9521153F4108F47BC078C0EC0180
:1022E000C11586E5D807E8F5C11525E5D20748F000
:1022F0008C2F0E9409108F7190E0982F8827906290
:1023000068C0C11534E5D30728F09C2F8827846F57
:10231000906A5FC0AE01437055272C2F26952695F5
:10232000C115D34578F481E090E002C0880F991F71
:102330004A95E2F740E2249F90011124822B932BCF
:102340009C6847C081E090E002C0880F991F4A95C1
:10235000E2F740E2249F90011124822B932B9A688C
:1023600038C0C1152AE5D207F8F4C11539E5D307FD
:1023700090F08C2F8F700E94091094E0D695C7952D
:102380009A95E1F7CF70D0E0DC2FCC27D0699E0181
:10239000282BC9011EC0C11548E5D407C0F09C2FE9
:1023A0008827806F906A15C0CE01905681159042A3
:1023B00070F48D2F8F710E940910282F2F71CE017C
:1023C00099279062922B05C081E090E002C080E0E6
:1023D00090E0DF91CF910895CF9384E090E00E9448
:1023E000012FC82F82E290E00E94012F2C2F30E0B5
:1023F000A901582BCA01CF91089569EE7EEF80E0C4
:1024000090E00E94432F60E082E090E00E94252F40
:1024100060E083E090E00E94252F10923704109234
:1024200038041092390410923A0460E084E090E09D
:102430000E94252F60E082E290E00E94252F60E05C
:1024400085E090E00E94252F60E086E090E00E9409
:10245000252F6FEF87E090E00E94252F40E050E0AD
:10246000BA0188E090E00E94372F60E08DE090E0B4
:102470000E94252F40E050E0BA0188E190E00E94E0
:10248000372F60E087E190E00E94252F40E050E088
:10249000BA018CE190E00E94372F60E070E080E2AA
:1024A00090E00E94432F40E050E0BA0188E190E0C4
:1024B0000E94372F40E050E0BA018FE090E00E9488
:1024C000372F40E050E0BA0183E190E00C94372FC1
:1024D0008091360481111092360408958095909170
:1024E00035048923809335040895909135048091B3
:1024F0003404982B9093BB03809136048823D9F041
:10250000892B8093BB0380910701882331F0809150
:10251000AD0587FF02C08EE101C086E0EDEBF3E080
:1025200090E0815028F021912223D9F39F5FF9CFC9
:1025300091110E94681240E250E064E174E08BEB7C
:1025400093E00E94FC2F892B21F180E2EBEBF3E07A
:10255000A4E1B4E001900D928A95E1F7E091A40521
:10256000F091A5053097A9F080910701882359F0D3
:102570008091AD0587FF07C08091BB038093BC03AA
:1025800086E08093BB030280F381E02D8BEB93E028
:102590000994089520911304809582238093130455
:1025A000982F977099F430E0482F082E000C550BA7
:1025B0002417350759F09091AE0592FD07C0859517
:1025C000859585950E94112B109213040895CF9341
:1025D000C091AE05C2FB992790F9981799F080FB3E
:1025E000C2F9C093AE056091AD0584E090E00E9411
:1025F000252F6C2F82E290E00E94252F82E0CF9160
:102600000C94CA12CF910895809112049091E10325
:10261000891719F08F5F8770FBCF08950F931F9371
:10262000CF93DF938091E00382958F7009F05DC0B6
:102630008091DD03882309F458C080911204109121
:10264000E1036091DB037091DC03C091DE03D09164
:10265000DF0391E06F3F09F090E0292F06E081173A
:1026600009F443C0209721F07F3F21F030E003C000
:1026700031E001C0322F90E030FD34C0089FF001FE
:10268000099FF00D1124DF01AE51BC4F11963C9112
:102690001197371327C03C91361324C012963C91F2
:1026A000129731111FC013964D915C9114974C1BDA
:1026B0005D0B483C5105B0F48091E0038F70806160
:1026C0008093E003E951FC4F80818F7080618083AB
:1026D0008BED93E00E942104DF91CF911F910F9128
:1026E0000C94041301968770BACFDF91CF911F919C
:1026F0000F9108959F92AF92BF92CF92DF92EF9287
:10270000FF920F931F93CF93DF93CDB7DEB76197FF
:102710000FB6F894DEBF0FBECDBF8C0185E0F80187
:10272000DE011D9601900D928A95E1F7F801E28095
:102730009091DB036091DC034091DE035091DF0355
:102740004115510531F06F3F31F481E09F3F19F49D
:1027500003C081E001C080E0F82FF1709F2E80FD62
:102760001AC1F80130812181C380D4808BEDA82E5D
:1027700083E0B82EF090DD03F601E41BF50BFF209B
:1027800009F4C6C08091E003E83CF10508F091C06F
:10279000482F407F09F050C0621311C093130FC03F
:1027A000FE2CE1100CC08F7080618093E003C501A6
:1027B0000E9421048091E003F801858329C1CD287E
:1027C00031F02F3F31F481E03F3F19F403C081E045
:1027D00001C080E080FD03C081E08E2502C080E062
:1027E00090E0F82FF170FF2E80FF1CC08091120442
:1027F0004091E10356E0841709F4E8C090E0589F47
:10280000F001599FF00D1124EE51FC4F6181261308
:1028100006C06081631303C06281E61203C00196A3
:102820008770E9CFFE2CEE2009F4F2C08091E0031E
:1028300081608093E00349C0621306C0931304C013
:10284000E11002C0F80186C0C8010E94612B8823F4
:1028500051F1EE2041F12091E003822F82958F709B
:1028600090E0029774F08091DB039091DC039887ED
:102870008F831986DB86CA862C87CE0107960E9435
:10288000210486E0F801ABEDB3E001900D928A954A
:10289000E1F70E940E130AC06217C9F0C8010E9436
:1028A000612B81111EC0C8010E942104FF24F394F2
:1028B000AFC0482F407F81F78BED93E00E94210449
:1028C00086E0F50111928A95E9F7F12CA1C09313E6
:1028D000E5CFE110E3CFF8018583C8010E94210410
:1028E00054C0EE2001F32091E003822F82958F7077
:1028F00090E0029734F28091DB039091DC039A839D
:1029000089831B82DD82CC822E83CE010196B7CFD4
:10291000E83CF105D0F5FE2CEE2029F2621327C029
:10292000931325C02091E00320FD18C0822F8295CB
:102930008F70482F50E04115510581F0F801258333
:102940004F30510541F08F5F982F9295907F822FE5
:102950008F70892B8583C8010E94210486E0F801CD
:10296000ABEDB3E001900D928A95E1F751C0C8013B
:102970000E94612B811185CF8091E003816080935B
:10298000E003C8010E94210443C086E0F5011192D2
:102990008A95E9F73DC0EE2009F485CFC8010E9471
:1029A000612BF82E882309F47ECF86E0F801ABED89
:1029B000B3E001900D928A95E1F78091DB0390914D
:1029C000DC030E94942A0E940E1322C03D872E87AA
:1029D0008D859E850E94942A292F22952F70223062
:1029E00028F49F7039F0811105C00BC0243028F401
:1029F0009F7049F4805E883020F0C8010E94210455
:102A00009F2CF92C05C0F8019581907F99F7F9CF9B
:102A10008F2D61960FB6F894DEBF0FBECDBFDF914C
:102A2000CF911F910F91FF90EF90DF90CF90BF90CB
:102A3000AF909F9008958F929F92AF92BF92CF9246
:102A4000DF92EF92FF920F931F93CF93DF93CDB757
:102A5000DEB72A970FB6F894DEBF0FBECDBFAE012A
:102A60004F5F5F4F7A018AE0DA011D928A95E9F79C
:102A700001E612E0CC24C394D12CAA24A394B12C57
:102A80004E01BBE08B0E911CF80180818F3F09F451
:102A90004AC0F894E82FE295EF70F0E021A18F7022
:102AA000A50102C0440F551F8A95E2F7CA01922F73
:102AB000982B91A392A18095892382A3789400C03A
:102AC0006FE672E0F701A60140955095DB012D916C
:102AD000BD012F3FA9F0822F82958F7090E0DC011D
:102AE00090968C9190E02F7002C0959587952A95CD
:102AF000E2F780FD05C0808191818C299D2904C069
:102B000080819181842395239183808332968E16D0
:102B10009F06E1F6F80180818F3F11F00E944C1072
:102B2000F0EAFA95F1F7CC0CDD1C0F5F1F4F42E085
:102B30000F36140709F0A8CF4AE050E0B7018CEE39
:102B400095E00E94FC2F11E0009709F410E0892B1A
:102B500089F08AE0F701ACEEB5E001900D928A951C
:102B6000E1F781E080933D040E94B71990933C0403
:102B700080933B0480913D04882391F180913B0434
:102B800090913C040E94A819059750F18091EC05A2
:102B90009091ED059093FC058093FB058091EE05E7
:102BA0009091EF059093FE058093FD058091F005CF
:102BB0009091F105909300068093FF058091F205B6
:102BC0009091F30590930206809301068091F4059D
:102BD0009091F505909304068093030610923D04AE
:102BE000812F2A960FB6F894DEBF0FBECDBFDF91BE
:102BF000CF911F910F91FF90EF90DF90CF90BF90FA
:102C0000AF909F908F900895089508958091B40596
:102C100008958093AF057093B1056093B0058091DE
:102C2000D705843001F582E08093E9008FEF909121
:102C3000E800815095FD06C095ED9A95F1F70000EA
:102C40008111F5CF8091E80085FF0DC040E050E094
:102C500063E070E08FEA95E00E94651D8091E800D6
:102C60008E778093E8000895BC0184E00C940916E7
:102C7000BC0183E00C940916CF93DF9320910701E8
:102C8000222339F02091AD0527FF03C060E222E046
:102C900002C068E021E02093E9002FEF3091E800C6
:102CA000215035FD06C035ED3A95F1F700002111B0
:102CB000F5CF2091E80025FF1DC0EC0180910701B0
:102CC000811105C040E050E068E070E003C070E0B2
:102CD00040E050E0CE010E94651D8091E8008E77B3
:102CE0008093E80080E2FE01A5EBB5E001900D9233
:102CF0008A95E1F7DF91CF910895FF920F931F938B
:102D0000CF93DF9300D000D0CDB7DEB780349105EC
:102D100088F5122F042FF62EBC01660F771F660F61
:102D2000771F605E7E4F44E050E0CE0101960E9426
:102D3000E82E898183704A81282F30E050E9859FF1
:102D4000C00111248C5A9B4FFC01E40FF11DB49774
:102D5000F0824B81FC01E40FF11DB49700834C819C
:102D6000840F911DFC01B4971083F901EE5AFB4FBB
:102D700081E080830F900F900F900F90DF91CF91A3
:102D80001F910F91FF900895FF920F931F93CF9380
:102D9000DF93182F062FF42EC0E0D0E02F2D402F08
:102DA000612FCE010E947D162196C034D105B1F766
:102DB000DF91CF911F910F91FF9008951F920F9275
:102DC0000FB60F9211242F933F934F935F936F93FE
:102DD0007F938F939F93AF93BF93CF93DF93EF93A3
:102DE000FF93C091E900CF708091EC00D82FD17093
:102DF00080FDD0E81092E9008091F000877F8093F9
:102E0000F00078940E94911D1092E9008091F000EA
:102E100088608093F000CD2BCF70C093E900FF91C4
:102E2000EF91DF91CF91BF91AF919F918F917F9162
:102E30006F915F914F913F912F910F900FBE0F9027
:102E40001F901895E8EDF0E080818E7F80831092CE
:102E5000E2001092DA001092E100A0EEB0E08C9156
:102E600081608C9380818F77808319BCA7EDB0E05F
:102E70008C918E7F8C9380818F7E80831092B2059F
:102E800008952091E4003091E50095E64091EC0032
:102E9000842F817040FF23C08091E80080FD1DC019
:102EA0008091D705882399F0853099F08091EB00C7
:102EB00085FD11C04091E4005091E50024173507CD
:102EC00029F3915011F09A01E1CF84E0089582E056
:102ED000089583E0089581E0089580E00895409189
:102EE000E80042FFDDCF08958091D90587FF11C02A
:102EF0008091E80082FD05C08091D7058111F8CF4F
:102F000011C08091E8008B770BC08091D705882392
:102F100049F08091E80080FFF8CF8091E8008E773B
:102F20008093E8000895982F973068F59093E90012
:102F3000981739F07091EC002091ED005091F0005D
:102F400003C0242F762F50E021FD02C09F5FECCFFD
:102F50003091EB003E7F3093EB003091ED003D7FF0
:102F60003093ED003091EB0031603093EB007093C3
:102F7000EC002093ED005093F0002091EE0027FD2F
:102F8000E5CF80E008958F708093E90081E0089597
:102F9000CF92DF92EF92FF920F931F93CF93DF9325
:102FA000C8EDD0E088818F7E8883E7EDF0E08081F6
:102FB0008160808384E082BF81E08093B205888154
:102FC0008E7F888302EE10E0F80110821092DA0002
:102FD00081EEC82ED12CF601108288818F778883EC
:102FE00088818068888388818F7D888319BC10924E
:102FF000D7051092D8051092D6051092D50590EEFF
:10300000E92EF12CF70180818B7F8083888181609C
:10301000888342E060E080E00E949317F60180819F
:103020008E7F8083F80180818160808380818860C9
:103030008083F70180818E7F80838881806188838F
:10304000DF91CF911F910F91FF90EF90DF90CF9084
:1030500008951F920F920FB60F9211242F933F9352
:103060004F935F936F937F938F939F93AF93BF9390
:10307000EF93FF938091E10082FF09C08091E2000D
:1030800082FF05C08091E1008B7F8093E1008091F9
:10309000DA0080FF2AC08091D80080FF26C080918E
:1030A000DA008E7F8093DA008091D90080FF18C00B
:1030B00080E189BD82E189BD09B400FEFDCF81E0D8
:1030C0008093D7058091B20581110FC00E9422170D
:1030D0000E94C8178091E20084608093E20005C0DE
:1030E00019BC1092D7051092B2058091E10080FFC3
:1030F00017C08091E20080FF13C08091E2008E7FB4
:103100008093E2008091E20080618093E2008091F0
:10311000D80080628093D80019BC85E08093D705E1
:103120008091E10084FF30C08091E20084FF2CC0D8
:1031300080E189BD82E189BD09B400FEFDCF8091A7
:10314000D8008F7D8093D8008091E1008F7E80939E
:10315000E1008091E2008F7E8093E2008091E200A6
:1031600081608093E2008091D805882311F084E08B
:1031700007C08091E30087FD02C081E001C083E0C9
:103180008093D7058091D7058091E10083FF27C008
:103190008091E20083FF23C08091E100877F8093CC
:1031A000E10082E08093D7051092D8058091E1007C
:1031B0008E7F8093E1008091E2008E7F8093E20019
:1031C0008091E20080618093E20042E060E080E074
:1031D0000E9493178091F00088608093F000FF9127
:1031E000EF91BF91AF919F918F917F916F915F917F
:1031F0004F913F912F910F900FBE0F901F901895F8
:103200002091DF053091E0052617370748F061155A
:10321000710539F42091E8002E772093E80001C071
:10322000B901FC0120E06115710579F18091D705A4
:103230008823F1F18530F1F18091E80083FD3CC0F5
:103240008091E80082FD2EC08091E80080FFEBCFE6
:103250002091F3008091F20090E0922B61157105AE
:1032600051F08830910538F421912093F10061509C
:1032700071090196F3CF21E0089709F020E08091D1
:10328000E8008E778093E800CECF2111CFCF0AC01F
:103290008091D705882361F0853061F08091E80046
:1032A00083FD0AC08091E80082FFF2CF80E008959C
:1032B00082E0089583E0089581E0089581E080939D
:1032C000E00080E28093D8001092C9008FE19EE474
:1032D0000197F1F700C0000087E090EBDC018093DC
:1032E0007F0690938006A0938106B09382069CE0AF
:1032F00088E10FB6F894A895809360000FBE909374
:103300006000FFCF78941F920F920FB60F92112496
:103310008F939F93AF93BF938091A9059091AA0536
:10332000A091AB05B091AC050196A11DB11D809394
:10333000A9059093AA05A093AB05B093AC05BF91E6
:10334000AF919F918F910F900FBE0F901F90189586
:103350009C014FB7F8948091A9059091AA05A0917E
:10336000AB05B091AC054FBF821B930B08952FB7EF
:10337000F8948091A9059091AA05A091AB05B09110
:10338000AC052FBF08951F920F920FB60F92112414
:103390008F939F93AF93BF938091A805811113C022
:1033A0008091A9059091AA05A091AB05B091AC05BB
:1033B0004196A11DB11D8093A9059093AA05A093E4
:1033C000AB05B093AC05BF91AF919F918F910F90DA
:1033D0000FBE0F901F901895209107012223C9F06E
:1033E0002091AD0527FF15C0262F269526952695F9
:1033F0002E31C8F4FC01E20FF11D677081E090E00E
:1034000001C0880F6A95EAF78095928189238283AB
:103410000895FC0106962281621301C01282319642
:10342000E817F907C1F70895209107012223C1F099
:103430002091AD0527FF14C0262F269526952695A9
:103440002E3130F5FC01E20FF11D677081E090E054
:1034500001C0880F6A95EAF79281892B82830895CB
:10346000FC0132962FEF30E04191641789F02F3F35
:1034700019F4411101C0232F3F5F3630A9F72F3FC8
:1034800039F0FC01E20FF11D27FDFA9562830895E2
:1034900008952091A6053091A7052817390771F0E6
:1034A0009093A7058093A605E091A405F091A5054A
:1034B000309721F00084F185E02D09940895209142
:1034C000A2053091A3052817390771F09093A30541
:1034D0008093A205E091A405F091A505309721F015
:1034E0000680F781E02D09940895E091A405F091FC
:1034F000A505309721F00190F081E02D099480E03E
:103500000895EF92FF920F93CF93DF93C42FD22FA2
:10351000FC0182818823D1F04093A1050E94B71954
:103520009093A00580939F0580E28C0F883008F06F
:103530006DC0C77081E001C0880FCA95EAF7DF91BE
:10354000CF910F91FF90EF900C949D2B8091A1054E
:1035500048134BC080919F059091A0050E94A81927
:10356000883C910508F041C0CD17C9F080E28C0F6E
:10357000883040F4C77081E001C0880FCA95EAF72F
:103580000E94962B80E28D0F883048F481E09D2FB9
:10359000977001C0880F9A95EAF70E949D2B093316
:1035A00019F0E12CF12C03C080E5E82EF12C802FDE
:1035B0000E94D12BE114F10451F08FE99FE00197B3
:1035C000F1F700C0000091E0E91AF108F3CF802F75
:1035D0000E94A72B80E28D0F8830C0F4D77081E065
:1035E00001C0880FDA95EAF70AC080E28C0F8830B4
:1035F00068F4C77081E001C0880FCA95EAF7DF91CF
:10360000CF910F91FF90EF900C94962BDF91CF917B
:103610000F91FF90EF90089590919A0590FF04C04C
:103620009695981740F003C0811105C090E0961759
:1036300010F40C94252A61E00C94DA29882311F007
:10364000FA0101C0FB010994DF92EF92FF920F9300
:103650001F93CF93DF93262F30E0A90148565A4F8E
:103660007A01FA01908191110AC0F7011082DF916D
:10367000CF911F910F91FF90EF90DF900895D82E7A
:10368000F2E16F9FE001112400E010E0F801EC0F7F
:10369000FD1FEC58FA4F4081602F8D2D0E94212D87
:1036A0000F5F1F4F0231110589F7DFCFCF93DF93F3
:1036B000C82F4BE06DEF0E94212D40E06AE08C2F77
:1036C0000E94212D8FE39CE90197F1F700C00000D3
:1036D00040E060E08C2F0E94212D40E061E08C2FC3
:1036E0000E94212D40E066E08C2F0E94212D40E0B9
:1036F0006DEF8C2F0E94212DD0E040E06D2F8C2F9C
:103700000E94212DDF5FD231C1F740E06D2F8C2F59
:103710000E94212DDF5FD432C1F740E06D2F8C2F46
:103720000E94212DDF5FD43BC1F74BE06DEF8C2F62
:103730000E94212D41E06AE08C2F0E94212D40E063
:103740006DEF8C2FDF91CF910C94212D0F931F9350
:10375000CF93DF93082F000FEB0114E210933E0488
:10376000EFE3F4E0DE018D91819384E0EF34F8071C
:10377000D1F724E630E041E150E06EE374E0802FC1
:103780000E94512E105F6096143B41F7DF91CF915C
:103790001F910F9108959091E605937071F08093B9
:1037A000E7056093E8054B3A08F04AEA4093E905DB
:1037B0008091E50581608093E5050895DF92EF92A1
:1037C000FF920F931F93CF93DF938C01C091080159
:1037D0008DE0C89FC02D1124DDE0DC0FD13408F04E
:1037E000D0E46091EA056695669521E0620F08F4E1
:1037F0006FEF8091E1059091E2050E947927D82E24
:10380000CD17F0F4EC2EF12CF701EF5DFD4F908118
:1038100080910901892391F06091E7057091E80595
:103820008091E9052D2D4C2FF80109950E943B2828
:10383000462F282F672FC7010E94A826CF5FE0CF11
:1038400081E0D03408F080E0DF91CF911F910F919B
:10385000FF90EF90DF9008959F92AF92BF92CF922A
:10386000DF92EF92FF920F931F93CF93DF936C0140
:10387000C09108018DE0C89FC02D1124DDE0DC0F50
:10388000D13408F0D0E46091EA05669566958091A0
:10389000E1059091E2050E947927182F80E4810FBD
:1038A0000E94C52690E8F92EF80E812F0E94C526A9
:1038B00020E8922E980ECD1700F5AC2EB12CF50114
:1038C000EF5DFD4F9081809109018923A1F0609106
:1038D000E7057091E8058091E905E12E0C2F292D6F
:1038E0004F2DF60109950E943B28462F282F672F60
:1038F000C5010E94A826CF5FDECF81E0D03408F05A
:1039000080E0DF91CF911F910F91FF90EF90DF90BA
:10391000CF90BF90AF909F9008956F927F928F92BB
:103920009F92AF92BF92CF92DF92EF920F931F932D
:10393000CF93DF933C01C09108018DE0C89FC02D5B
:103940001124DDE0DC0FD13408F0D0E46091EA0509
:1039500066958091E1059091E2050E947927182FE4
:10396000CD1708F044C08C2E912CF401EF5DFD4F73
:103970009081809109018923C1F1F401EE0FFF1FAD
:10398000EF55FE4FC080D12C80E7C81AD108F40152
:10399000EE0FFF1FEE55FE4FA080B12CE0E2AE1AF5
:1039A000B108CC9C9001CD9C300D300D1124AA9C07
:1039B000C001AB9C900D900D1124820F931F0E94AB
:1039C0001F27082F6091E7057091E8058091E905B0
:1039D000E12E9501A601F30109950E943B28462F8F
:1039E000282F672FC4010E94A826CF5FB9CF81E09E
:1039F000D03408F080E0DF91CF911F910F91EF90CC
:103A0000DF90CF90BF90AF909F908F907F906F90FE
:103A10000895CF92DF92EF92FF920F931F93CF936F
:103A2000DF936C01C09108018DE0C89FC02D112467
:103A3000DDE0DC0FD13408F0D0E46091EA05669552
:103A40008091E1059091E2050E947927182FCD170A
:103A500078F5EC2EF12CF701EF5DFD4F9081809110
:103A60000901892319F1F701EE0FFF1FEE55FE4FF3
:103A7000208130E020523109F701EE0FFF1FEF5592
:103A8000FE4F408150E0405751096091E705709129
:103A9000E8058091E905012FF60109950E943B2870
:103AA000462F282F672FC7010E94A826CF5FCFCFB0
:103AB00081E0D03408F080E0DF91CF911F910F9129
:103AC000FF90EF90DF90CF900895EF92FF920F93C9
:103AD0001F93CF93DF937C018B010E9441178111CB
:103AE00019C0E70101151105A1F08091E80085FDDD
:103AF0000AC08091E8008E778093E8000E94411709
:103B0000882381F307C089918093F1000150110946
:103B1000E9CF80E0DF91CF911F910F91FF90EF905F
:103B200008951F93CF93DF93CDB7DEB7AA970FB653
:103B3000F894DEBF0FBECDBFE9EDF5E081EE95E074
:103B40002091F10021938E179F07D1F78091DA051C
:103B5000833009F461C030F4813071F0823009F4AF
:103B60009BC0B2C08A3009F487C08B3009F46CC0A6
:103B7000893009F0A9C020C08091D905813A09F0A7
:103B8000A3C08091E800877F8093E8008091DD05E5
:103B90009091DE05892B21F460E285EB95E003C06E
:103BA00060E080E090E070E00E9400198091E80001
:103BB0008B778093E80088C08091D905813209F025
:103BC00083C08091DD059091DE05029708F07CC0EE
:103BD0008091E800877F8093E8008091E80082FD73
:103BE00005C08091D7058111F8CF6EC02091F300F8
:103BF0008091F20090E0922B029731F48091F100D5
:103C0000813011F0863021F48091F1008093B40569
:103C10008091E8008B7754C08091D905813A09F0F2
:103C200053C08091DD059091DE05892B09F04CC0D1
:103C30008091E800877F8093E8008091E80080FF12
:103C4000FCCF8091070137C08091D9058132E1F521
:103C50008091DD059091DE05892BB1F58091E8001A
:103C6000877F8093E8000E9474178091DB05809322
:103C700007010E94812B28C08091D905813221F54E
:103C80008091E800877F8093E8000E9474178091FC
:103C9000DC058093B30518C08091D905813AA1F461
:103CA0008091E800877F8093E8008091E80080FFA2
:103CB000FCCF8091B3058093F1008091E8008E776E
:103CC0008093E8000E9474178091E80083FFCEC1C2
:103CD0008091D9059091DA05492F50E04A3051057D
:103CE00008F0C4C1FA01EA57FF4F0C94CE2F803878
:103CF00021F0823809F0BAC108C08091D5059091B1
:103D0000D605992389F082600FC08091DD058F7000
:103D1000873008F0ABC18093E9008091EB0085FB10
:103D2000882780F91092E9009091E800977F90939E
:103D3000E8008093F1001092F10065C1282F2D7FDB
:103D400009F094C1882319F0823061F08FC180910D
:103D5000DB05813009F08AC1933009F080E080935F
:103D6000D6052EC08091DB0581112AC08091DD052A
:103D70008F702FEF280F263008F078C18093E9006C
:103D80002091EB0020FF1CC0933021F48091EB00C8
:103D9000806214C09091EB0090619093EB0021E061
:103DA00030E0A90102C0440F551F8A95E2F7409305
:103DB000EA001092EA008091EB0088608093EB00AB
:103DC0001092E9008091E800877F20C181114EC1E7
:103DD0001091DB051F778091E3008078812B809321
:103DE000E3008091E800877F8093E8000E947417C9
:103DF0008091E80080FFFCCF8091E3008068809391
:103E0000E300111102C082E001C083E08093D70576
:103E10002DC18058823008F029C18091DB05909136
:103E2000DC058C3D53E0950779F583E08A838AE2CF
:103E300089834FB7F894DE01139620E03EE051E20B
:103E4000E32FF0E050935700E49120FF03C0E29588
:103E5000EF703F5FEF708E2F90E0EA3010F0C79662
:103E600001C0C0968D939D932F5F243149F74FBFBA
:103E70008091E800877F8093E8006AE270E0CE01DD
:103E800001960E940019AEC04091DD055091DE05FB
:103E9000292F332723303105A9F068F4213031056B
:103EA00009F4F3C02230310509F0E0C08BE390E063
:103EB000EDECF2E044C02132310521F1223231052E
:103EC00071F1D4C0992781309105A1F058F0029783
:103ED00009F0CCC0EAE1F3E0E4918E2F90E0EAE152
:103EE000F3E02AC0EAE4F3E0E4918E2F90E0EAE404
:103EF000F3E022C0EEE2F3E0E4918E2F90E0EEE2F8
:103F0000F3E01AC04115510509F4C4C04130510510
:103F100009F0ACC089E090E0E8EFF2E010C0411594
:103F2000510509F4BCC04130510509F09FC08DE630
:103F300090E0E0E2F2E003C0009709F497C020911E
:103F4000E800277F2093E8002091DF053091E0050D
:103F50008217930708F49C0140E02115310589F18F
:103F60008091D705882309F43DC08530D9F180912F
:103F7000E80083FD37C08091E80082FD2FC080916A
:103F8000E80080FFEACF4091F3008091F20090E0DA
:103F9000942B2115310559F08830910540F4449156
:103FA0004093F1003196215031090196F2CF41E062
:103FB000089709F040E08091E8008E778093E80050
:103FC000CCCF4111CDCF0AC08091D705882351F0C5
:103FD000853041F08091E80083FD04C08091E800C5
:103FE00082FFF2CF8091E8008B778093E8003EC09B
:103FF0008038E1F58091E800877F8093E800809128
:10400000D8058093F1008091E8008E778093E800D6
:104010000E9474172BC0811129C08091DB059091FB
:10402000DC059927029714F58091E800877F80933B
:10403000E8001091DB051093D8050E947417111148
:1040400006C08091E30087FD02C081E001C084E0EA
:104050008093D70542E061EC81E00E94931742E231
:1040600061EC82E00E9493178091D7058091E8006F
:1040700083FF1AC08091E800877F8093E8008091D9
:10408000EB0080628093EB000FC082E190E0E8E0FB
:10409000F3E055CF89E090E0EFEDF2E050CF80E41F
:1040A00090E0EDE8F2E04BCFAA960FB6F894DEBFB1
:1040B0000FBECDBFDF91CF911F910895CF93DF93B6
:1040C000CDB7DEB72A970FB6F894DEBF0FBECDBFCF
:1040D00084B7877F84BF0FB6F894A895809160005D
:1040E000886180936000109260000FBE90E080E8CD
:1040F0000FB6F89480936100909361000FBE85B76E
:10410000806885BF85B7806885BF87E090E1909320
:10411000A3028093A2020E9422170E94C8178091D6
:10412000E20084608093E20078948091D705882330
:10413000A1F01091E9001F709091EC00892F81701F
:1041400090FD80E8182B1092E9008091E80083FD33
:104150000E94911D1F701093E90082E084BD93E0DE
:1041600095BD9AEF97BD80936E0001E612E0D801ED
:104170008D918D018F3F11F00E944C10B2E00F36EF
:104180001B07A9F70FE612E0F4E7EF2EF2E0FF2E8F
:10419000F80181918F018F3F11F00E944C10E016C1
:1041A000F106B1F78AE0EBEFF5E0DF01282F1D9271
:1041B0002A95E9F7ECEEF5E0DF011D928A95E9F723
:1041C00080E090E00E940F2F893E9E4F11F00E94E8
:1041D000FD1182E090E00E94012F809305060E946D
:1041E000EC119093AE058093AD050E941B15EFE393
:1041F000FCE93197F1F700C000000E941B15809187
:10420000FB0580FF08C06FEF7FEF80E090E00E9429
:10421000432F0E945E1983E090E00E94012F682FD7
:1042200070E080E090E00E94572B0E945B2C80E0C1
:1042300090E00E940F2F893E9E4F21F00E94FD11B9
:104240000E94AA2646E050E06CE170E086EE95E020
:104250000E94F12E1092E5058091E6058C7F11F405
:104260000E94AA268091FA05811136C080E090E074
:104270000E940F2F893E9E4F21F00E94FD110E9447
:104280002B2888E090E00E94092F60939A05709394
:104290009B0580939C0590939D056E7F71F40E9411
:1042A0002B2888E090E00E94092F60939A05709374
:1042B0009B0580939C0590939D050E94DD2710929D
:1042C000510680919A0580FF04C060E086950E94A7
:1042D000DA2981E08093FA058BE091E09093A505BF
:1042E0008093A40558E1C52ED12C60E4962E75E08C
:1042F000A72E76E0B72EE0E18E2E8091D70585308F
:1043000009F043C012E18091D705853009F039C02A
:104310008091D705843019F10E94CE0A1092A80529
:104320000FB6F894A895C09260000FBE90926000FE
:1043300083B7817F846083BF83B7816083BF7894B4
:10434000889583B78E7F83BF0FB6F894A895809128
:104350006000886180936000109260000FBE8091C1
:10436000D605882309F4CFCF0E941B15EBEFF5E0AB
:1043700081919191892B09F00EC1AE16BF06C1F74C
:10438000C2CF0E94812B0E94751A0E941B158823A0
:1043900059F08FB7F8944091A9055091AA05609102
:1043A000AB057091AC058FBFABEFB5E0E6E0F6E092
:1043B00000E010E0702F2D913D9181919191822725
:1043C0009327009779F160E0EE24E394F12CAC019F
:1043D0004E215F21452B09F169837A832E213F21EC
:1043E00081E0232B09F480E08B830E94B719816060
:1043F000782F9D838C8349815A816B818D810E94A6
:104400007903000F111FF801EA5FF94F8081918154
:10441000E826F926F182E0821AC06F5FEE0CFF1CDD
:104420006E30A9F60F5F1F4F0530110519F68FEF9B
:104430008E838F8318860E94B7198160782F9A87A0
:1044400089874E815F8168858A850E947903809182
:104450005106882309F493C080915006E0919A0593
:10446000E695E81BE0934C06823059F4F0E0E45AFC
:10447000FC4FE4910E2F10E0E2E9EE2EE6E2FE2E74
:1044800059C0863059F4F0E0E75AFC4FE4910E2F02
:1044900010E072E8E72E76E2F72E4CC0893061F426
:1044A000E695F0E0EA5AFC4FE4910E2F10E065E14A
:1044B000E62E66E2F62E3EC08F3061F4E695F0E01F
:1044C000ED5AFC4FE4910E2F10E055EAE52E55E22F
:1044D000F52E30C0853159F4F0E0E05BFC4FE491FB
:1044E0000E2F10E044E5E42E45E2F42E23C088317F
:1044F000A1F0833249F4EEE4F3E00591149132E443
:10450000E32E36E2F32E16C0843271F404EF11E08C
:104510002BE8E22E24E2F22E0DC008E210E098EC27
:10452000E92E94E2F92E06C000ED17E08AE8E82EA5
:1045300084E2F82E80914D06882361F010924D069A
:104540000E94B71990934B0680934A0610924F062B
:1045500010924E060E94B719E0914A06F0914B0660
:104560008E1B9F0B8F3F9F4750F40E0F1F1F109302
:104570004B0600934A068AE496E0F70109950E94EB
:10458000CE0A0E94751A90911006891709F4B5CECB
:1045900080931006B2CE89BC19BD09B400FEFDCFD0
:1045A0008091D8008F7D8093D8008091E000826058
:1045B0008093E0008091E00081FDFCCF0E94812B80
:1045C000A2CEE42FF0E0EE0FFF1FEF55FE4F9081DB
:1045D000921B97FD9195292F38E1239F212D1124BE
:1045E000620F08950F931F9310E0F801EE0FFF1F65
:1045F000EF55FE4F9081905797FD9195000F111F39
:10460000F801EE55FE4FE081F0E0B097DF01AA0F10
:10461000BB1F8D010E0F1F1F2003D001219FB00D66
:104620001124E8E3F0E0E91BF10997FDF3959F0100
:10463000220F331F89010E0F1F1F40039001419F5E
:10464000300D11242A0F3B1F37FF02C021583F4F66
:10465000220F232F221F330B620F1F910F910895FA
:104660000F931F93522F10E0F801EE0FFF1FEE552E
:10467000FE4FE081F0E0B097EE0FFF1F9F01520365
:10468000D001539FB00D1124000F111FF801EF55F9
:10469000FE4F008110E000571109000F111F400369
:1046A0009001419F300D11242A0F3B1F37FF02C09C
:1046B00021583F4F220F232F221F330B620F1F91D0
:1046C0000F9108950F931F93522F10E0F801EE0FF2
:1046D000FF1FEE55FE4FE081F0E0B0979F015203BF
:1046E000D001539FB00D1124000F111FF801EF5599
:1046F000FE4F008110E00057110940039001419FD7
:10470000300D11242A0F3B1F37FF02C021583F4FA5
:10471000220F232F221F330B620F1F910F91089539
:10472000EF920F931F9393E0099F80011124159539
:1047300007956E2D600F1F910F91EF900895A22F96
:1047400050E0FA01EE0FFF1FEE55FE4F90819052A0
:1047500097FD9195440F551FFA01EF55FE4F30819B
:10476000232F30E02A1B3109290F311D97FD3A957F
:10477000620F0895E42FF0E0EE0FFF1FEE55FE4F9D
:104780006081621B0895E42FF0E0EE0FFF1FEF55EC
:10479000FE4F6081621B0895622F0895E42FF0E0C0
:1047A000EE0FFF1FEF55FE4F408134EE439F412D2A
:1047B0001124E72FF0E050E0445E5F4FDA01A21BC6
:1047C000B1099D01B7FF03C031952195310993E0EF
:1047D000220F331F9A95E1F7AF01421B530B9A0149
:1047E00057FF02C020E030E0279F212D1124722FB7
:1047F0000895FC019B01009721F477FF2BC080E80E
:104800000895AC0197FF04C044275527481B590B56
:10481000B901640F751F37FD0CC0241B350BC9018E
:10482000A5E0880F991FAA95E1F70E94BA2F80E2B0
:104830000CC0CB0165E0880F991F6A95E1F7BA01BA
:10484000621B730B0E94BA2F80E6861BF7FF03C022
:104850008195089580E00895EF920F93CF93DF93B1
:10486000D72FC82FC9010E19BA010E94F923602F52
:10487000681B7D2F8C2FDF91CF910F91EF900895C2
:104880000F93CF93DF93D72FC82FC901BA010E948E
:10489000F923682F600F7D2F8C2FDF91CF910F911F
:1048A0000895EF920F931F93CF93DF93D62F172F77
:1048B000C82FC9010E19070FBA010E94F923702FE2
:1048C000781B719F712D11246D2F8C2FDF91CF914B
:1048D0001F910F91EF900895FF920F931F93CF9325
:1048E000DF93F62E172FD82FC901C72FC01BBA018F
:1048F0000E94F923982F990F890F7C2F781B719FA5
:10490000712D11246F2D8D2FDF91CF911F910F915C
:10491000FF9008950895EF92FF920F931F93CF9306
:10492000DF938C01C4E1D6E0E12CF12CF801848105
:10493000F9E0EF16F1041CF4882351F002C0811154
:1049400007C040919D05413808F040E89E0102C033
:104950009E0140E060919C0580919B050E94CB28C0
:104960008FEFE81AF80A239692E1E916F104F1F6BE
:104970000E949627F801848190E001968170992722
:104980008483DF91CF911F910F91FF90EF90089555
:104990008F929F92AF92BF92CF92DF92EF92FF924F
:1049A0000F931F93CF93DF93EC014C81042F10E002
:1049B0009801D8010E949D2F9B01AC010E94682F95
:1049C0006B017C01E0E2F0E0E01BF10BA5E5B0E05B
:1049D0009B01AC010E94682F4B015C019F01DF012C
:1049E0000E94D42F9B01AC010E94732F9B01AC014C
:1049F0002C0D3D1D4E1D5F1DC501B4010E947B2F76
:104A0000822FF22E99E2921728F093E0299F9001CD
:104A100011240DC025E530E0281B3109C901880F9C
:104A2000991F280F391F37FF02C02F5F3F4F359561
:104A30002795122F109594E1C92E96E0D92E00E00B
:104A400085E5E82EEF1801FD02C08E2D01C08F2DE7
:104A5000412F113808F040E8960160919C050E94B2
:104A6000CB280F5F83E0C80ED11C023161F70E9492
:104A700096278C81811102C091E003C0803219F425
:104A80009FEF9093190190911901890F8C83DF9109
:104A9000CF911F910F91FF90EF90DF90CF90BF903B
:104AA000AF909F908F9008950F931F93CF93DF93B4
:104AB000C4E1D6E0FE01118210821282339686E0B4
:104AC000EA34F807C1F700E010E080911206082EE2
:104AD000000C990B08171907ACF080911801082EEB
:104AE000000C990B801791076CF040919D0541389F
:104AF00008F040E89E0160919C0580919B050E9412
:104B0000CB2803C0198218821A820F5F1F4F239689
:104B100002311105D1F60E949627809117019091DC
:104B20001206980F9093120620911801280F2093D7
:104B30001801121614F491311CF08195809317011D
:104B4000DF91CF911F910F910895BF92CF92DF9285
:104B5000EF92FF920F931F93CF93DF93FC0182811B
:104B600080FF03C0DD24DA9402C0DD24D39404E185
:104B700016E0C0E0D0E022E1B22EF80111821082EE
:104B8000128294E0E92EF12CC12C809111068C0D3B
:104B900083312CF06B2D0E94AC2F892F02C087FD32
:104BA0008E5E082E000C990BC817D907A9F48091C6
:104BB0009D058E9DA0018F9D500D11245595479503
:104BC00055954795413808F040E8980160919C055B
:104BD00080919B050E94CB28CD0CF1E0EF1AF108E3
:104BE000A1F621960D5F1F4FC231D10531F60E940B
:104BF00096278091110691E0D91206C0811102C05A
:104C000081E107C0815005C090E00196BE010E947D
:104C1000BA2F80931106DF91CF911F910F91FF90D2
:104C2000EF90DF90CF90BF900895EF92FF921F9387
:104C3000CF93DF93EC0184E1E82E86E0F82E10E0BC
:104C400040919D05413808F040E88C8197016091C2
:104C50009C05810F0E94CB28125F83E0E80EF11CB7
:104C60001C3F71F70E9496279A818C8190FF02C0A9
:104C70008F5F01C081508C83DF91CF911F91FF9096
:104C8000EF9008950F931F93CF93DF9300D01F925F
:104C9000CDB7DEB78C018091130681110AC09E0149
:104CA0002F5F3F4F40E86FEF0E94CB288A818093AF
:104CB0001306F8018481813051F028F0823061F4CC
:104CC000409113060AC08091130640E007C060912E
:104CD000130640E080E003C040E080E060E00E9416
:104CE000CC27F801848190E0019663E070E00E9497
:104CF000BA2F84830F900F900F90DF91CF911F9167
:104D00000F910895CF93DF93EC01EAE9F5E0438139
:104D100062818C810E94D9288C818F5F8C83DF9186
:104D2000CF910895CF93DF93EC01EC81F0E0E05A4E
:104D3000FC4F4491EAE9F5E0628181810E94D92823
:104D40008C818F5F8C83DF91CF9108950C94C41672
:104D50000C947D16E6EEF5E089E2808380912701D0
:104D600090912801A091290181839283A3838FE7E9
:104D700084838FEF858346E050E06CE170E0CF01E3
:104D80000E94152F1092E5050895482F982F46FD93
:104D90009095E92FEF739F7046FD9F5FE295EF704E
:104DA000EE0FF0E0EC58FD4F2181299F802D212D41
:104DB000112482958F702295207F822B3081982F2D
:104DC000930F892F47FD8195805808950F931F9366
:104DD000CF93DF93D62F072F182FC42F822F0E9437
:104DE000C526EC2FF0E0EE0FFF1FEF55FE4F908130
:104DF0009058890F87FD8195880F682F2CE0629F5E
:104E0000612D11246D0F702F812FDF91CF911F9194
:104E10000F91089540911A0150911B0125E038E04F
:104E2000429FC001439F900D529F900D1124875EB9
:104E3000994C90931B0180931A01890F0895BC012E
:104E40008230910508F40895613E8EE1780748F4B8
:104E50009B0195E0369527959A95E1F748E0420F3A
:104E600001C04FEF91E0242F30E0290F311D35951F
:104E70002795229FF001239FF00DF00D11246E174E
:104E80007F0718F44FEF420F04C02F3F39F091E035
:104E9000920F491740F78FEF890F08958FEF08950C
:104EA0000F93CF93DF93D72FC82F47FD4195E8E3AA
:104EB000F0E0CF01841B910947FD9395889FB001D5
:104EC000899F700D700D1124229FC001239F900DAA
:104ED000900D1124860F971F0E941F27682F660FC1
:104EE000860F682F600F7D2F8C2FDF91CF910F9150
:104EF000089520E030E0869F212D969F200D311DE2
:104F00001124C90108952091EA0530E1230F08F426
:104F10002FEF60E1822F90E00E947927BC0188EB9F
:104F20009BE00E94782E80E090E0089580919A05A1
:104F300080FF0AC0579A8BB18F779BB190682FB7CB
:104F4000F894E4E1F6E00BC0E4E1F6E011821082AF
:104F50001282339636E0EA34F307C1F7EBCF36E03E
:104F6000EA34F30789F0319148E09BB9000000C0B2
:104F700037FF8BB9330F000000C000C000C08BB9F1
:104F800000C04A9591F7EBCF2FBF8FE594E00197D2
:104F9000F1F700C00000089590919A0590FF0CC0B1
:104FA000E4E1F6E0818360834283339696E0EA345D
:104FB000F907C1F70C949627089580919A05282F38
:104FC000269530E02115310519F48170826005C005
:104FD0002532310524F08170886480939A05809190
:104FE0009D05813818F080E880939D050895CF9243
:104FF000DF92EF92FF926B017C010E94DD27B701E7
:10500000A60188E090E0FF90EF90DF90CF900C94A5
:10501000372F80919E05882319F0815080939E053B
:1050200060919A0570919B0580919C0590919D05DA
:105030000C94F72780919E05833018F48F5F80933E
:105040009E0560919A0570919B0580919C059091B9
:105050009D050C94F727EAE9F5E083E0808311824F
:105060008FEF828380E883831482608171818281E3
:1050700093810C94F727CF92DF92EF92FF920F93D8
:105080001F93CF93DF93F62E472FE82FF0E0711197
:1050900006C0E05AFB4F8491782F682F73C0272FEA
:1050A00030E0E05AFB4FE491FE2F0E2F10E056E067
:1050B000659FC0011124CFEFD0E0BE010E94782E81
:1050C0005BEA5603C001579F900D11248F0D911D6F
:1050D0008F0D911D982F990F980F7E01E21AF30AF8
:1050E000E09ED001E19EB00DF09EB00D11248B2FFB
:1050F000499FA0011124452F55277E01E41AF50A86
:10510000E09EA001E19E500DF09E500D11246E0115
:10511000C91AD108C29E7001C39EF00CD29EF00C39
:1051200011242F2D3327C21BD30BC09F9001C19F89
:10513000300DD09F300D1124932F6230710591F006
:1051400048F461157105E1F061307105B9F49E2FE5
:10515000E52F16C06430710569F040F066307105C6
:1051600079F00CC09E2FEB2F832F0AC0EB2F8F2FCF
:10517000952F06C09B2F8E2FE32F02C09B2F852FCC
:105180007E2F692FDF91CF911F910F91FF90EF90AC
:10519000DF90CF900895CF93DF93762FE901682FAA
:1051A000842F0E943B28798368838A83DF91CF9183
:1051B0000895CF93DF9300D01F92CDB7DEB79091C3
:1051C0009A0590FF0DC0413808F040E89E012F5F1E
:1051D0003F4F0E94CB284B8169818A810E94CC2756
:1051E0000F900F900F90DF91CF9108955F926F9283
:1051F0007F928F929F92AF92BF92CF92DF92EF9267
:10520000FF920F931F93CF93DF9300D01F92CDB7E0
:10521000DEB7082F762E142F622E90919A0590FFFC
:1052200074C0E92FE695AE2FB0E0A458BD4F8C9125
:10523000809350069E7F923081F4413808F040E818
:105240009E012F5F3F4F672D802F0E94CB284B81FF
:1052500069818A810E94CC2746C0823019F410915E
:105260009D0541C0863019F400919B053CC08930F2
:10527000D9F38931C1F5E9518E2F8170582EE69509
:10528000F0E0E05AFA4FA590B49084E1C82E86E091
:10529000D82EE12CF12CBB2492E1892E912CAE9CCE
:1052A000C001AF9C900DBE9C900D1124B4010E94D2
:1052B000782E802F511002C0860F01C0861B412F0F
:1052C000113808F040E89601672D0E94CB288FEF37
:1052D000E81AF80A83E0C80ED11C82E1E816F1044E
:1052E000F1F60E94962700939B0570929C051093FF
:1052F0009D05662051F060919A0570919B05809103
:105300009C0590919D050E94F7270F900F900F909C
:10531000DF91CF911F910F91FF90EF90DF90CF9091
:10532000BF90AF909F908F907F906F905F90089507
:10533000EAE9F5E0438128E0421B08F440E021E07F
:10534000628181810C94F628EAE9F5E0438128E046
:10535000420F08F44FEF21E0628181810C94F6281E
:10536000EAE9F5E0628128E0621B08F460E021E0F0
:10537000438181810C94F628EAE9F5E0628128E016
:10538000620F08F46FEF21E0438181810C94F628CD
:10539000EAE9F5E0818121E04381628188500C9443
:1053A000F628EAE9F5E0818121E043816281885FA6
:1053B0000C94F62890919A0590FF3DC09170811150
:1053C00002C0926006C0853210F0986402C0880F57
:1053D000982B90939A05662351F060919A057091ED
:1053E0009B0580919C0590919D050E94F7276091F7
:1053F0009A05669570E04BE050E08CE191E00E94E8
:10540000EF2F892B19F01092510609C081E080938B
:1054100051060E94B71990934B0680934A0681E08B
:1054200080934D0620E040919D0560919C05809100
:105430009B050C94F628089580919A0586958150D5
:1054400009F484E261E00C94DA2980919A0586954A
:105450008F5F853208F081E061E00C94DA2980E00A
:1054600090E00E945F1A80E090E00E94491A10923A
:1054700034040C9475128F929F92AF92BF92DF9278
:10548000EF92FF920F931F93CF93DF938090F605D7
:105490009090F705A090F805B090F9054091370479
:1054A000509138046091390470913A04842A952A05
:1054B000A62AB72ACFE1D0E02EE0929F70011124F6
:1054C00096E4D92E082F10E0D501C4010C2E04C09B
:1054D000B695A795979587950A94D2F780FD04C055
:1054E000219790F780E014C0DC9EF001DD9EF00D66
:1054F0001124EE0DFF1DE00FF11FEE0FFF1FEB5902
:10550000FA4F859194910E946310019749F38C2F73
:10551000DF91CF911F910F91FF90EF90DF90BF909F
:10552000AF909F908F900895CF93DF93EC010E94EE
:105530003B2A26E4829FC0011124FC012EE0D29F69
:10554000E00DF11D1124EC0FF11DEE0FFF1FEB59C3
:10555000FA4F859194910E946310DF91CF91089545
:105560002EE0929F800D1124682F669566956695B2
:10557000982F977085E0689FB001112440E050E0BB
:1055800080E0FB01E40FF51FEE5AF94F208130E077
:10559000092E02C0369527950A94E2F72170332729
:1055A000042E01C0220F0A94EAF7822B4F5F5F4F4F
:1055B0004530510531F708952EE0929F800D11245A
:1055C000E82FE695E695E695877051E001C0550F06
:1055D0008A95EAF785E0E89FF0011124EE5AF94F29
:1055E00020E030E070E04081CB01022E02C09695B1
:1055F00087950A94E2F78170819584278523842713
:1056000081932F5F3F4F2530310569F708956093EF
:10561000F6057093F7058093F8059093F9050C94BF
:105620002F2A0F931F9341E050E060E070E004C028
:10563000440F551F661F771F8A95D2F740955095E6
:10564000609570958091F6059091F705A091F80509
:10565000B091F9058A019B01082319232A233B23D2
:10566000C901B8011F910F910C94072B0F931F9341
:1056700041E050E060E070E004C0440F551F661F39
:10568000771F8A95D2F78091F6059091F705A09142
:10569000F805B091F9058A019B01082B192B2A2BDB
:1056A0003B2BC901B8011F910F910C94072B6093FC
:1056B0003704709338048093390490933A040C941F
:1056C0002F2AFC01808191810E94942A92959F70DB
:1056D000963079F010F4925001C09A50923068F4EC
:1056E000803F69F018F4883E40F409C0843F29F4F3
:1056F00006C0883E20F0813F11F080E0089581E0EF
:1057000008951092350480910701882331F080912B
:10571000AD0587FF02C08EE101C086E0EDEBF3E04E
:10572000DF011D928A95E9F70C942F2A882321F036
:105730000E946E120C9475120895882339F090918E
:105740003504892B809335040C94751208958823B1
:1057500039F1682F8CEF860F813A28F48BEB93E0B8
:105760000E94EC190CC080E2860F883050F46770FC
:1057700081E001C0880F6A95EAF70E946E120C94CE
:1057800075128BE5860F833020F480E090E00C9456
:105790005F1A685A673120F480E090E00C94491A4F
:1057A0000895CF93882309F46DC09CEF980F913A28
:1057B000C8F5C82F809107018823E1F08091AD05DD
:1057C00087FF18C0EC2FE695E695E695F0E0E554E6
:1057D000FC4F8281282F30E04C2F477081E090E011
:1057E00002C0880F991F4A95E2F782239323892BE1
:1057F00061F412C0EDEBF3E083EC93E02191C2176A
:1058000021F08E179F07D1F707C06C2F8BEB93E029
:105810000E94EC190E9475126C2F8BEB93E00E9492
:10582000141A13C090E2980F983090F4877021E01A
:1058300030E0A90102C0440F551F8A95E2F7CA0162
:1058400090913504892B80933504CF910C94751277
:10585000EBE5E80FE33040F4F0E0E65DFE4F8081D9
:1058600090E0CF910C945F1A885A873158F4E82F52
:10587000F0E0EE0FFF1FE35DFE4F80819181CF913D
:105880000C94491ACF91089580915204882329F0ED
:1058900064E574E084E70E94A61B10925204809194
:1058A0005304882329F064EE74E087E70E94A61B66
:1058B0001092530408956F927F928F929F92AF92AD
:1058C000BF92CF92DF92EF92FF920F931F93CF93ED
:1058D000DF9300D000D0CDB7DEB70E949A2D84E7C9
:1058E0000E94561B87E70E94561B00E211E072E1FE
:1058F000772EE8E0CE2ED12CEE24E394F12C662412
:10590000639444E050E0B801CE0101960E94E82E75
:105910002A8130E0C9018497AB80B12C44E2A41AFB
:10592000B108EC81F0E0B497AC0197FF02C0495F89
:105930005F4F63E0559547956A95E1F7298123709C
:1059400030E0729EB001739E700D11246C587A4F36
:105950004B01840E911CB6010E94BA2FD70102C0E0
:10596000AA0FBB1F8A95E2F7CD01D4019C91892B28
:105970008C93C501B7FC079653E0959587955A958A
:10598000E1F7729EA001739E500D11244C585A4F9E
:105990004A01880E911CC501B6010E94BA2FA701C9
:1059A00002C0440F551F8A95E2F7CA01D4019C91A9
:1059B000892B8C93CF01F7FD079643E0959587954A
:1059C0004A95E1F7729EA001739E500D11244C5828
:1059D0005A4F5A01A80EB11CCF01B6010E94BA2F2E
:1059E000F70102C0EE0FFF1F8A95E2F7CF01D50144
:1059F0009C91892B8C93F901E856FA4F60820C5FD9
:105A00001F4FB2E000321B0709F07BCF60E084E754
:105A10000E94241B61E087E70E94241B0F900F90D7
:105A20000F900F90DF91CF911F910F91FF90EF900A
:105A3000DF90CF90BF90AF909F908F907F906F90AE
:105A40000895EEE3F4E06083418324E630E042E031
:105A500050E0BF01880F0C94512E1F93CF93DF931A
:105A6000FC01EF5DFD4F20816223D1F0EC010E942B
:105A7000D82E182F0E94D82E8F77782F20E8720FFB
:105A800008F47FEF612F8091E9050E943B28462FA3
:105A9000282F672FCE01DF91CF911F910C94A8265C
:105AA000DF91CF911F910895DF92EF92FF920F93B4
:105AB0001F93CF93DF93EC01FC01EF5DFD4F9081CD
:105AC000692381F1D090E8050091E9051091E7057F
:105AD000E12EF12C0E94D82E282FC7018C549F4F05
:105AE00068E671E00E94BA2F8E199F0997FD039610
:105AF00095958795959587952370612F289F600DC3
:105B000011247D2D802F0E943B28462F282F672FA0
:105B1000CE01DF91CF911F910F91FF90EF90DF9019
:105B20000C94A826DF91CF911F910F91FF90EF90D9
:105B3000DF9008951092B9008CE08093B80008952A
:105B40009F92AF92BF92CF92DF92EF92FF920F930C
:105B50001F93CF93DF93B82EEB010E94B7196C010E
:105B6000C431D10558F0CF3F8FEFD80759F0CE019F
:105B700064E170E00E94782E7B0107C0EE24E3947C
:105B8000F12C03C025E0E22EF12C84E8A82E94EA43
:105B9000992E1092BC009092BC000E94B7198C0103
:105BA0008091BC0087FD08C00E94B719801B910B33
:105BB0008E159F05A8F32AC08091B900887F883090
:105BC00041F08091B900887F803119F00FEF1FEF0D
:105BD0001FC0B092BB00A092BC000E94B7198C01FC
:105BE0008091BC0087FD08C00E94B719801B910BF3
:105BF0008E159F05A8F30AC08091B900887F88316F
:105C000011F0803419F700E010E00EC00EEF1FEF26
:105C1000CF3F8FEFD80709F4BCCFC6010E94A81967
:105C20008C179D0708F4B5CFC801DF91CF911F9164
:105C30000F91FF90EF90DF90CF90BF90AF909F902B
:105C400008950F931F93CF93DF93EB018093BB00D5
:105C500084E88093BC000E94B7198C018091BC003D
:105C600087FD0EC0CF3F8FEFD807C1F30E94B71951
:105C7000801B910B8C179D0788F38EEF9FEF0CC054
:105C80002091B900287F81E090E0283211F480E073
:105C900090E0919581959109DF91CF911F910F919E
:105CA0000895CF92DF92EF92FF920F931F93CF93BD
:105CB000DF936B018A017901B9010E94A02DE601F1
:105CC0000C0D1D1DC017D10761F424E92093BC0001
:105CD000DF91CF911F910F91FF90EF90DF90CF90C8
:105CE000089597FDF2CFB70189910E94212EEACF46
:105CF000AA1BBB1B51E107C0AA1FBB1FA617B707F2
:105D000010F0A61BB70B881F991F5A95A9F780950D
:105D10009095BC01CD0108958F929F92AF92BF9252
:105D2000CF92DF92EF92FF92CF93DF93EC016881E5
:105D300079818A819B81611571058105910521F425
:105D400064E279ED8BE597E02DE133EF41E050E03F
:105D50000E94492F49015A019B01AC01A7EAB1E415
:105D60000E94682F6B017C01ACEEB4EFA501940199
:105D70000E94762FDC01CB018C0D9D1DAE1DBF1D39
:105D8000B7FF03C00197A109B04888839983AA830C
:105D9000BB839F77DF91CF91FF90EF90DF90CF9003
:105DA000BF90AF909F908F9008950E948C2E089581
:105DB00080E091E00E948C2E0895A0E0B0E08093F6
:105DC000000190930101A0930201B0930301089593
:105DD000FB01DC0102C005900D9241505040D8F704
:105DE0000895DC01CB01FC01F999FECF06C0F2BD9C
:105DF000E1BDF89A319600B40D9241505040B8F789
:105E00000895F999FECF92BD81BDF89A992780B582
:105E10000895A6E1B0E044E050E00C94F32EA8E130
:105E2000B0E042E050E00C94F32EDC01A40FB51F6B
:105E30004150504048F0CB01840F951F2E910E9495
:105E4000262F41505040D0F70895262FF999FECFC4
:105E500092BD81BDF89A019700B4021639F01FBABD
:105E600020BD0FB6F894FA9AF99A0FBE08950396DA
:105E7000272F0E94262F0E94252F252F0E94262F94
:105E8000242F0C94262F0196272F0E94262F0C9446
:105E9000252F052E97FB1EF400940E94602F57FDBE
:105EA00007D00E947B2F07FC03D04EF40C94602F88
:105EB00050954095309521953F4F4F4F5F4F089536
:105EC00090958095709561957F4F8F4F9F4F089566
:105ED0000E949D2FA59F900DB49F900DA49F800DB3
:105EE000911D11240895B7FF0C94682F0E94682F0C
:105EF000821B930B0895A1E21A2EAA1BBB1BFD0166
:105F00000DC0AA1FBB1FEE1FFF1FA217B307E40798
:105F1000F50720F0A21BB30BE40BF50B661F771FF0
:105F2000881F991F1A9469F76095709580959095D0
:105F30009B01AC01BD01CF010895A29FB001B39FA9
:105F4000C001A39F700D811D1124911DB29F700D82
:105F5000811D1124911D089587FB082E062687FDBB
:105F6000819567FD61950E94E32F0EF4919507FCE2
:105F70008195089597FB072E16F4009407D077FDBE
:105F800009D00E94782E07FC05D03EF490958195AB
:105F90009F4F0895709561957F4F0895EE0FFF1FF5
:105FA0000590F491E02D09940E949D2F332312F463
:105FB0008A1B9B0B0C94DE2F0E949D2FB7FF089528
:105FC000821B930B0895991B79E004C0991F9617C3
:105FD00008F0961B881F7A95C9F780950895FC01F3
:105FE0004150504030F001900616D1F73197CF0163
:105FF0000895882799270895FB01DC0104C08D913D
:106000000190801921F441505040C8F7881B990B2A
:066010000895F894FFCF93
:1060160001000000FFFF030100FF0006163C160505
:1060260016381634160416010201390501191A1B11
:106036001C1D1E1F20212200FFAA818283E200E987
:1060460000EA00B500B600B700CD008301CC008A97
:10605600019201940121022302240225022602272D
:10606600022A02B300B4006F007000121314151652
:106076001718101124252627281A1B1C1D1E1F1948
:1060860030292A2B2C2D2E080700202122233132DD
:10609600333435FF2F09FF0A010203040538373967
:1060A6003A3B360E0D0C0BFFFF060FFFFF3C3D3E45
:1060B6003F302030304030503060307030704020FB
:1060C600201020103020304040284014400040006E
:1060D60000100020003000400050006000601000FA
:1060E600101010201030104010501040205020602A
:1060F600207020700080009000A000B000C000D08A
:1061060000E00080109010A010B010C010D810D879
:1061160020701080209020A020B020C020E0309079
:10612600308030A030B030C030A040B440C840E02D
:1061360040040404040404040401010401010101EF
:10614600010404040404040401040404040404040F
:106156000404040404040404010104040404040102
:1061660001040404040404010404040401010101FB
:10617600016766363534F7F6F5C63092949593F096
:10618600F1F43796003131295A1B750A00010202D3
:1061960002020606060909090909090F0F0F0F0F62
:1061A6000F15151518191919191919191919192366
:0261B6002400C3
:00000001FF
